:100000000C9473000C949B000C949B000C949B002C
:100010000C949B000C9472070C949B000C949B0016
:100020000C949B000C949B000C949B000C949B00E4
:100030000C949B000C949B000C949B000C949B00D4
:100040000C940A050C949B000C941C040C94F6036D
:100050000C949B000C949B000C949B000C949B00B4
:100060000C9454050C949B001F0C210C230C250CA4
:10007000270C290C2B0C2D0C5F0C620C650C5C0CF6
:10008000680C6B0C7C0C7C0C00000000240027002A
:100090002A0000000000250028002B0000000000BE
:1000A00023002600290004040404040404040202BA
:1000B00002020202030303030303010204081020E7
:1000C00040800102040810200102040810200000F2
:1000D0000008000201000003040700000000000007
:1000E00000003B20132011241FBECFEFD8E0DEBF5D
:1000F000CDBF24E0A8EFB1E001C01D92A933B20743
:10010000E1F711E0A0E0B1E0ECE1FFE402C005900E
:100110000D92A83FB107D9F710E0C2E7D0E004C0C4
:100120002197FE010E94C123C137D107C9F70E9460
:1001300050150C9481270C9400000895CF92DF9203
:10014000EF92FF920F931F93CF93DF936C017A018D
:100150008B01C0E0D0E0CE15DF0589F0D8016D91AC
:100160008D01D601ED91FC910190F081E02DC60149
:100170000995892B11F47E0102C02196ECCFC701AD
:10018000DF91CF911F910F91FF90EF90DF90CF9073
:100190000895FC01918D828D981761F0828DDF01A9
:1001A000A80FB11D5D968C91928D9F5F9F73928F6A
:1001B00090E008958FEF9FEF0895FC01918D828D5F
:1001C000981731F0828DE80FF11D858D90E008952C
:1001D0008FEF9FEF0895FC01918D228D892F90E084
:1001E000805C9F4F821B91098F739927089586EF3A
:1001F00092E00E94EB0021E0892B09F420E0822F9D
:100200000895FC01848DDF01A80FB11DA35ABF4FD3
:100210002C91848D90E001968F739927848FA68905
:10022000B7892C93A089B1898C9180648C93938D2C
:10023000848D981306C00288F389E02D80818F7D1C
:1002400080830895EF92FF920F931F93CF93DF93D4
:10025000EC0181E0888F9B8D8C8D981305C0E88917
:10026000F989808185FD24C0F62E0B8D10E00F5F8B
:100270001F4F0F731127E02E8C8DE8120CC00FB6A4
:1002800007FCFACFE889F989808185FFF5CFCE0197
:100290000E940101F1CF8B8DFE01E80FF11DE35AA1
:1002A000FF4FF0820B8FEA89FB898081806207C053
:1002B000EE89FF896083E889F98980818064808381
:1002C00081E090E0DF91CF911F910F91FF90EF902F
:1002D0000895CF93DF93EC01888D8823C9F0EA89D4
:1002E000FB89808185FD05C0A889B9898C9186FD2F
:1002F0000FC00FB607FCF5CF808185FFF2CFA8892C
:10030000B9898C9185FFEDCFCE010E940101E7CF25
:10031000DF91CF91089580E090E0892B29F00E9431
:10032000F70081110C9400000895833081F028F4C7
:10033000813099F08230A1F008958730A9F088309B
:10034000B9F08430D1F4809180008F7D03C080911A
:1003500080008F7780938000089584B58F7702C0E6
:1003600084B58F7D84BD08958091B0008F7703C0E0
:100370008091B0008F7D8093B0000895CF93DF937C
:10038000282F30E0F901E253FF4F8491F901E65440
:10039000FF4FD491F901EA55FF4FC491CC2391F05E
:1003A00081110E949501EC2FF0E0EE0FFF1FE45643
:1003B000FF4FA591B491EC91ED2381E090E021F401
:1003C00080E002C080E090E0DF91CF9108953FB7D8
:1003D000F8948091820290918302A0918402B0915E
:1003E000850226B5A89B05C02F3F19F00196A11DD7
:1003F000B11D3FBFBA2FA92F982F8827820F911DBB
:10040000A11DB11DBC01CD0142E0660F771F881F01
:10041000991F4A95D1F7089585ED8093BC0080918E
:10042000BC0084FDFCCF1092CE02089540915C0286
:10043000262F30E0240F311D21323105DCF42091CC
:10044000CE022430C9F4FC0180E090E0861758F415
:1004500030915C022191DC01A65CBD4FA30FB11D60
:100460002C930196F3CF80915C02680F60935C023D
:1004700080E0089581E0089582E008950895E09174
:10048000870280918602E81730F4F0E0E857FD4FCC
:10049000808190E008958FEF9FEF089590918702FB
:1004A00080918602981750F4E92FF0E0E857FD4F4D
:1004B000208130E09F5F9093870202C02FEF3FEFD3
:1004C000C90108958091860290E020918702821BE5
:1004D00091090895CF92DF92EF92FF920F931F93AD
:1004E000CF93DF937C01262F972F8A018091CF0233
:1004F000882391F0C62FD72F6E01C40ED51ECC15C0
:10050000DD0571F06991D701ED91FC910190F081C9
:10051000E02DC7010995F3CF642F822F0E941602A8
:10052000C801DF91CF911F910F91FF90EF90DF9065
:10053000CF900895CF93DF931F92CDB7DEB7698335
:100540002091CF022223D1F02091F102203240F0FD
:1005500021E030E0FC013383228380E090E015C08D
:100560008091D002E82FF0E0EF52FD4F9981908307
:100570008F5F8093D0028093F10205C061E0CE01CD
:1005800001960E94160281E090E00F90DF91CF91DA
:1005900008950E946327FC0180819181009711F0EA
:1005A0000C94222160E070E0CB0108950F931F931B
:1005B000CF93DF938C01EB01FC0180819181009747
:1005C000B1F0688179816115710579F042815381BB
:1005D0002C813D814217530740F00E947A278C817D
:1005E0009D81F8019583848313C00E940126888130
:1005F0009981F801918380838A819B81938382838F
:100600008C819D8195838483198218821B821A8232
:100610001D821C82DF91CF911F910F9108950F933E
:100620001F93CF93DF93EC0188819981009729F084
:100630002A813B812617370788F48B016F5F7F4F34
:100640000E949926009761F0998388831B830A830F
:100650002C813D81232B11F4FC01108281E001C02B
:1006600080E0DF91CF911F910F910895EF92FF925B
:100670000F931F93CF93DF93FC0124813581611584
:10068000710511F480E019C041155105A9F07B01F5
:10069000EC018A01020F131FB8010E940F03882387
:1006A00089F3288139818C819D81B701820F931F45
:1006B0000E947A271D830C8381E0DF91CF911F91E7
:1006C0000F91FF90EF900895CF93DF93EC01888115
:1006D0009981009711F00E940126198218821D82CB
:1006E0001C821B821A82DF91CF910895EF92FF92B4
:1006F0000F931F93CF93DF93EC017B018A01BA0123
:100700000E940F03811104C0CE010E94640307C040
:100710001D830C83B701888199810E947A27CE01BD
:10072000DF91CF911F910F91FF90EF900895CF939C
:10073000DF93EC016115710559F0FB010190002078
:10074000E9F73197AF01461B570B0E94760302C0B1
:100750000E946403CE01DF91CF910895CF93DF9380
:10076000EC01FB018617970761F0608171816115CB
:10077000710529F0448155810E94760302C00E94D0
:100780006403CE01DF91CF910895FC0180819181B6
:100790000C940126FC0111821082138212821582B0
:1007A00014826115710551F0FB0101900020E9F7F9
:1007B0003197AF01461B570B0C94760308956115D2
:1007C000710579F0FB0101900020E9F73197AF0145
:1007D000461B570BDC01ED91FC910280F381E02D6B
:1007E000099480E090E008950C94DF031F920F922B
:1007F0000FB60F9211242F933F934F935F936F93F4
:100800007F938F939F93AF93BF93EF93FF9386EF65
:1008100092E00E940101FF91EF91BF91AF919F91F2
:100820008F917F916F915F914F913F912F910F9099
:100830000FBE0F901F9018951F920F920FB60F9238
:1008400011242F938F939F93EF93FF93E0910603CF
:10085000F09107038081E0910C03F0910D0382FD7C
:1008600012C0908180910F038F5F8F7320911003CE
:10087000821751F0E0910F03F0E0EA50FD4F958FA1
:1008800080930F0301C08081FF91EF919F918F9121
:100890002F910F900FBE0F901F9018951F93CF931D
:1008A000DF93282F30E0F901E253FF4F8491F901E3
:1008B000E654FF4FD491F901EA55FF4FC491CC2380
:1008C000C9F0162F81110E949501EC2FF0E0EE0F78
:1008D000FF1FEE56FF4FA591B4918FB7F8941111F9
:1008E00005C09C91ED2FE095E92302C0EC91ED2B22
:1008F000EC938FBFDF91CF911F910895CF93DF933A
:10090000EC0160E08E810E944E0461E08E810E94C5
:100910004E0460E08E810E944E048BE891E00197C6
:10092000F1F7DF91CF910895CF93DF9390E0FC0131
:10093000E654FF4F2491FC01EA55FF4F8491882330
:1009400061F190E0880F991FFC01E857FF4FC591B6
:10095000D491FC01EE56FF4FA591B491611109C0ED
:100960009FB7F8948881209582238883EC912E2369
:100970000BC0623061F49FB7F8943881822F809564
:1009800083238883EC912E2B2C939FBF06C08FB7B7
:10099000F894E8812E2B28838FBFDF91CF910895A3
:1009A0008F929F92AF92BF92CF92DF92EF92FF927F
:1009B0006B017C010E94E7014B015C01C114D10471
:1009C000E104F104F1F00E94E701DC01CB01881998
:1009D0009909AA09BB09883E9340A105B10570F3A6
:1009E00021E0C21AD108E108F10888EE880E83E000
:1009F000981EA11CB11CC114D104E104F10419F723
:100A0000DDCFFF90EF90DF90CF90BF90AF909F90A1
:100A10008F9008951F920F920FB60F9211242F936B
:100A20003F938F939F93AF93BF938091FC019091DD
:100A3000FD01A091FE01B091FF013091810223E000
:100A4000230F2D3720F40196A11DB11D05C026E806
:100A5000230F0296A11DB11D209381028093FC01FA
:100A60009093FD01A093FE01B093FF01809182025B
:100A700090918302A0918402B09185020196A11DFC
:100A8000B11D8093820290938302A0938402B0935D
:100A90008502BF91AF919F918F913F912F910F90C0
:100AA0000FBE0F901F9018951F920F920FB60F92C6
:100AB00011242F933F934F935F936F937F938F9363
:100AC0009F93AF93BF93EF93FF938091B900887F7B
:100AD000803609F49CC068F5883209F45BC090F454
:100AE000803109F454C038F4882309F4F6C0883002
:100AF00009F44DC0F6C0883109F44CC0803209F4C5
:100B00005DC0EFC0803409F468C048F4803309F454
:100B100055C0883309F0E5C08093CC02D8C0803539
:100B200009F44FC0883509F45DC0883409F0D9C094
:100B3000D6C0883909F4C7C0A8F4883709F467C05B
:100B400038F4883609F463C0803709F460C0C9C03E
:100B5000883809F4B8C0803909F45FC0803809F0DA
:100B6000C0C05BC0803B09F486C038F4803A09F409
:100B700066C0883A09F47FC0B4C0803C09F4A7C0BD
:100B8000883C09F4A4C0883B09F48AC0AAC08091BB
:100B9000A90210C09091CB028091CA02981770F5FB
:100BA000E091CB0281E08E0F8093CB02F0E0E6551E
:100BB000FD4F80818093BB0085EC86C08093CC0282
:100BC0008EC0E091CB0281E08E0F8093CB028091AA
:100BD000BB00F0E0E655FD4F80839091CB02809101
:100BE000CA026EC0E091CB0281E08E0F8093CB02EF
:100BF0008091BB00F0E0E655FD4F80838091CD02EF
:100C000081116DC081E08093A80284EA61C083E015
:100C10008093CE0210928002CFCF809180028032EA
:100C200008F051C0E091800281E08E0F8093800235
:100C30008091BB00F0E0E05AFD4F8083BDCF85EC92
:100C40008093BC001092CE0280918002803230F4FA
:100C5000E0918002F0E0E05AFD4F10826091800246
:100C600070E0E0915E02F0915F0280E692E009950B
:100C70001092800236C084E08093CE0210925D0212
:100C800010925C02E0915A02F0915B02099580910A
:100C90005C02811105C081E080935C0210923A02EF
:100CA000E0915D0281E08E0F80935D02F0E0E65CF2
:100CB000FD4F80818093BB0090915D0280915C022A
:100CC000981708F479CF85E88093BC000AC085ECBA
:100CD0008093BC001092CE0204C01092CC020E94FD
:100CE0000C02FF91EF91BF91AF919F918F917F91F6
:100CF0006F915F914F913F912F910F900FBE0F9089
:100D00001F901895CF92DF92EF92FF920F931F934F
:100D1000CF93DF937C016C0187E0C80ED11CC0E04B
:100D2000D0E0062F10E0B8010C2E02C07595679533
:100D30000A94E2F76170F60181916F010E944E04FE
:100D40002196C430D10579F7C701DF91CF911F916A
:100D50000F91FF90EF90DF90CF900C947E04CF9294
:100D6000DF92EF92FF920F931F93CF93DF93EC01EB
:100D7000F62E642F8C810E944E048D818F3F19F0D6
:100D800060E00E944E048F850F2D10E084FF25C087
:100D90006E0187E0C80ED11CE12CF12CB8010E2C9D
:100DA00002C0759567950A94E2F76170F60181912A
:100DB0006F010E944E04FFEFEF1AFF0A88E0E81669
:100DC000F10461F7CE01DF91CF911F910F91FF9058
:100DD000EF90DF90CF900C947E04B80184E075957D
:100DE00067958A95E1F7CE010E9482066F2DCE01AC
:100DF000DF91CF911F910F91FF90EF90DF90CF90F7
:100E00000C94820641E00E94AF0681E090E00895D4
:100E100040E00C94AF06CF93DF9300D0CDB7DEB7A0
:100E200086EF92E00E94EB00892BB1F086EF92E012
:100E30000E94EB00892B81F086EF92E00E94C900AE
:100E400089831A8241E050E0BE016F5F7F4F87EED9
:100E500093E00E943603EACF0F900F90DF91CF917D
:100E600008950F931F9380910002813049F50E94ED
:100E70000A09FC0120910102309102024091030213
:100E8000509104026091F8017091F9018091FA018A
:100E90009091FB010E945C230081118122813381AA
:100EA000DC01CB01800F911FA21FB31F8093F202C0
:100EB0009093F302A093F402B093F5020E942309E9
:100EC0000E940A09FC0180819181A281B3818093F3
:100ED000F2029093F302A093F402B093F5021F91F3
:100EE0000F9108951F920F920FB60F9211242F9316
:100EF0003F934F935F936F937F938F939F93AF93A2
:100F0000BF93CF93DF93EF93FF938091F5030E94FC
:100F1000BE01EC018091F4030E94BE01CC0FDD1FE5
:100F20008C2BE091F303EF7094E0E99FF001112422
:100F3000E80FF11DE65FFE4F80818093F30380731D
:100F4000803161F48091010290910202A09103022C
:100F5000B09104020197A109B1090DC0803299F442
:100F60008091010290910202A0910302B0910402CB
:100F70000196A11DB11D8093010290930202A093DE
:100F80000302B0930402FF91EF91DF91CF91BF91E3
:100F9000AF919F918F917F916F915F914F913F9111
:100FA0002F910F900FBE0F901F901895382F209102
:100FB000F10290913404213208F049C08091CE02B0
:100FC0008111FCCF42E04093CE023093CD023FEF3F
:100FD0003093CC021092CB022093CA02A1EDB2E072
:100FE0004AEA52E0FA013E2F341B321718F43D91C1
:100FF0003193F9CF1092A9022091A902990F922B57
:101000009093A9029091A802913061F41092A802E5
:101010009091A9029093BB009091BC0093FDF8CFF2
:1010200095EC01C095EE9093BC009091CE02923069
:10103000E1F39091CC029F3F79F08091CC02803215
:1010400041F08091CC02803331F084E005C081E032
:1010500003C082E001C083E01092D0021092F1023E
:101060001092CF020895EF92FF920F931F93CF93A8
:10107000DF931F92CDB7DEB7162F91E09093CF028A
:1010800090E6909334041092D0021092F102682FEF
:1010900083E993E079830E949A02E12E7981F72E09
:1010A0008701085F1F4FF70161917F0183E993E09A
:1010B0000E949A02E016F106B1F781E00F90DF91ED
:1010C000CF911F910F91FF90EF900C94D607EF9264
:1010D000FF920F931F93CF93DF93EC01623018F0D0
:1010E0008F8588608F876B8B1C8A80E48D8B80E175
:1010F0008E8B80E58F8B61E08C810E9494048D81C2
:101100008F3F19F061E00E94940461E08E810E949B
:1011100094047E0187E0E80EF11C00E010E08F856A
:1011200084FD03C084E090E002C088E090E00817EE
:1011300019074CF461E0F70181917F010E9494044A
:101140000F5F1F4FECCF8BE39DE00197F1F760E05D
:101150008C810E944E0460E08E810E944E048D813D
:101160008F3F19F060E00E944E046F8564FD1DC042
:1011700063E0CE010E9482060BE416E4C8010197E9
:10118000F1F763E0CE010E948206C8010197F1F7F2
:1011900063E0CE010E94820683E592E00197F1F7B9
:1011A00062E0CE010E94820616C06062CE010E94FB
:1011B00008078BE496E40197F1F76F856062CE0132
:1011C0000E94080783E592E00197F1F76F8560625E
:1011D000CE010E9408076F856062CE010E94080759
:1011E00084E0888B6CE0CE010E94080761E0CE01AC
:1011F0000E9408078BE39FE10197F1F782E0898B5A
:1012000066E0CE01DF91CF911F910F91FF90EF909B
:101210000C9408070F931F93CF93DF9302EF12E014
:10122000CAE0D0E0CE010E94BF22F80181938F0175
:101230002196CE30D105B1F782EF92E0DF91CF91C8
:101240001F910F910895EF92FF920F931F93CF93E9
:10125000DF931F92CDB7DEB702EF12E08AE0E82EEF
:10126000F12CF80161918F01C70169830E94BF22AF
:101270006981681719F0C7010E94C722FFEFEF1AB2
:10128000FF0A8EE0E816F10461F782EF92E00F901A
:10129000DF91CF911F910F91FF90EF900895CF9321
:1012A000C62F91E09093CF0290E690933404109271
:1012B000D0021092F102682F83E993E00E949A0213
:1012C0006C2F83E993E00E949A0281E0CF910C9405
:1012D000D607CF93DF9391E09093CF0290E690935F
:1012E00034041092D0021092F102682F83E993E047
:1012F0000E949A0281E00E94D6078091CE0281115D
:10130000FCCF91E09093CE021092CD028FEF8093AC
:10131000CC021092CB021092CA029093A902909133
:10132000A902906C9093A9028091A802813061F487
:101330001092A8028091A9028093BB008091BC000A
:1013400083FDF8CF85EC01C085EE8093BC008091D1
:10135000CE028130E1F38091CB02811103C0C091B4
:10136000CB0201C0C1E0AAEAB2E028E832E0F9010C
:101370008E2F821B8C1718F48D918193F9CF1092C8
:101380008702C093860280918702C81731F083E9F3
:1013900093E00E944E02D82FF6CF8D2FDF91CF9190
:1013A00008952F923F924F925F926F927F928F9209
:1013B0009F92AF92BF92CF92DF92EF92FF920F93E4
:1013C0001F93CF93DF93CDB7DEB763970FB6F89433
:1013D000DEBF0FBECDBF322E3A874B875C876D874D
:1013E000272E2C011F870E876091300470913104E5
:1013F000809132049091330424E630E040E050E0E4
:101400000E942F242A8B3B8B4D835E83762E672E82
:10141000888B998B80912A0490912B04A0912C04A5
:10142000B0912D046C017D01FF0CCC08DC2C760101
:101430009C01AD016C2D7C2D8C2D9C2D0FE10E940B
:10144000FA24A12CEAECBE2EFAE9CF2EABE3DA2E79
:10145000E12CF12C00E010E00E945C24AA88BB88FB
:10146000CD80DE80E72CF62C088919890E94C723DD
:101470000FE10E94152549015A01D501C401BB0F96
:10148000880B982FDC0189839A83AB83BC839401FA
:10149000A5016981762F862F962FAA88BB88CD80DB
:1014A000DE80E72CF62C08890E94312539014A019B
:1014B000698B788B89839D83232D3A854B855C8549
:1014C0006D85722DC2012F3FA7E53A07A7E44A07B1
:1014D000A8EF5A07ADE06A07710581059105A9F0EB
:1014E000A0F0211534404B46544F644171058105ED
:1014F0009105B9F0B0F0312CA4E0AA87BBE6BB8718
:10150000E4EFEC87F4E1FD8709C0312CE8E5EA87D8
:10151000F7E4FB8788EF8C879DE09D87212C412C89
:10152000512C53016401E988F88809811D81232D1C
:101530003A854B855C856D85722DC2010E948D2494
:101540002E833F83488759878E819F81A885B985DF
:101550000F97A105B10558F49301A401B701C80183
:1015600004E00E94FA2409810E943A2528C08E8155
:101570009F81A885B9858B359105A105B10530F10D
:101580009301A4016989788989819D8102E00E9483
:10159000FA2453016401E988F88809811D810E94B9
:1015A0003A2559016A017B01E82F192F04E00E94B6
:1015B000FA240E2F0E943A2501E00E94FA24322ECE
:1015C0003A874B875C876D87272E2C015301640176
:1015D000E988F88809811D81232D3A854B855C8532
:1015E0006D85722DC2010E948B242901B42FA52F75
:1015F000F62FE72F382E292E05E00E94FA245201FB
:10160000CB2EDA2EEF2EFE2E032D122D0E943A2520
:1016100005E00E94FA24032D0E94312505E00E9476
:10162000FA24032D0E943A2519012A01B62FA72F6B
:10163000F82FE92F05E00E94FA2459016A017B0185
:101640008C019101A2016B2F7A2F8F2F9E2F0E9468
:10165000312553016401E988F88809811D810E94C0
:101660008D2469017A01C114D104E104F10429F443
:10167000812C912C5401839406C088248A94982C40
:101680003FE0A32EB12C87E0CC0CDD1CEE1CFF1C30
:101690008A95D1F7C701B601A50194010E94802364
:1016A0004E805F806884798497E0440C551C661CEA
:1016B000771C9A95D1F792E0591A61087108420E89
:1016C000531E641E751EC501B4010E945C23C61A18
:1016D000D70AE80AF90A84E190E00E946C258C019F
:1016E000DC019C9211968C921197862D8370129634
:1016F0008C93129713965C92139714964C92D50183
:10170000C4012CE0B695A795979587952A95D1F7B2
:10171000982F907F8E2D8F70882E890EF8018582EC
:10172000D682C7828E859F85892B19F4B8018AE1FC
:1017300006C0AE85BF85119721F4B80182E20E94F0
:101740003308C80163960FB6F894DEBF0FBECDBF55
:10175000DF91CF911F910F91FF90EF90DF90CF908D
:10176000BF90AF909F908F907F906F905F904F90C1
:101770003F902F900C9401262F923F924F925F92B0
:101780006F927F928F929F92AF92BF92CF92DF9291
:10179000EF92FF920F931F93CF93DF93CDB7DEB7F6
:1017A0002E970FB6F894DEBF0FBECDBF982E792EC0
:1017B00049875A876B877C876BA05C2C2D2C3E2D2C
:1017C000402E312EC984DA84EB84FC8484E190E0DD
:1017D0002E873D870E946C258C01FC01D082C1823E
:1017E000892D880F880F880F845D0E9469098C7F7E
:1017F0003D85932F9370892BF80182832382548235
:10180000D701C6016CE0B695A795979587956A951F
:10181000D1F7982F907F2E85822F8F70C82EC90EFA
:10182000C58236824782E92CF72CF8E0EF16F104E6
:10183000B8F4F701EC5CFF4FB8010C94C1238AE2C5
:101840000DC082E30BC08AE309C082E407C08AE4CA
:1018500005C082E503C08AE501C08BE50E9433081C
:1018600080E1980E892D0E94690991E0682FA912E4
:1018700002C0606401C06F7B892D0E944F09E1E0C6
:10188000EE16F10451F0F2E0EF16F10449F0E11424
:10189000F10449F4A092270412C0A092280412C0B7
:1018A000A092290412C088E0E816F104B0F4F70110
:1018B000E45CFF4F0C94C12354E4B52E0EC04CE2FF
:1018C000B42E0BC034E3B32E08C02CE3B22E05C0F7
:1018D0009CE4B92E02C084E5B82E8B2D0E946909C4
:1018E000837861108C6090E1899E40011124682FFB
:1018F00068298B2D0E944F09C8012E960FB6F894C7
:10190000DEBF0FBECDBFDF91CF911F910F91FF9032
:10191000EF90DF90CF90BF90AF909F908F907F908F
:101920006F905F904F903F902F900C9401262F92D4
:101930003F924F925F926F927F928F929F92AF925F
:10194000BF92CF92DF92EF92FF920F931F93CF93AC
:10195000DF93CDB7DEB76A970FB6F894DEBF0FBE40
:10196000CDBF322E232E4D875E873B012C01A982ED
:10197000B98ACA8ADB8AEC8AFD8A0E8B1F8B988A09
:101980008F86211500EA30070CEA400709EB500763
:1019900003E0600771058105910511F008F046C06C
:1019A0002F3F10EE310715EF410715E05107610594
:1019B00071058105910561F058F02F3F354D41418A
:1019C0005E47634071058105910509F0D8F50BC0AC
:1019D000312CB1EE2B2EF5EFFD8705E00E87612C43
:1019E000712C412C512C298139894A895B896C8958
:1019F0007D898E899F89A0E00E944C2509F0AEC0A8
:101A0000A32CB22CCD84DE847301820120E034E06B
:101A10004BE654EF64E170E080E090E00E948D249A
:101A200029873A874B875C87912C24C0312CF0EAB8
:101A30002F2E1CEA1D8729EB2E87A3E06A2E712C1E
:101A4000412C512C298139894A895B896C897D898E
:101A50008E899F89A0E00E944C2509F025C1992418
:101A6000939414E0E12EF12C00E010E0E986FA8670
:101A70000B871C87E984FA840B851C85A8019701D4
:101A800060E070E0CB01A32CB22CCD84DE84730126
:101A9000820129833A834B835C836D837E838F83AA
:101AA000988760E070E080E090E00E94C72329837F
:101AB000398B4A8B5B8B6C8B7D8B8E8B9F8BFF2442
:101AC000F3949F1409F4F3C010E0812C912C54017D
:101AD0008394C12CD12C760101C011E007E0CC0C1D
:101AE000DD1CEE1CFF1C0A95D1F7C701B601A5014C
:101AF00094010E94802389859A85AB85BC8567E027
:101B0000880F991FAA1FBB1F6A95D1F79250A10990
:101B1000B109820F931FA41FB51FEF85F889808339
:101B20009183A283B383C501B4010E945C23C61ACA
:101B3000D70AE80AF90AC482D582E682F78280864B
:101B40009186A286B3861111E5C0298139894A8917
:101B50005B896C897D898E899F89E2C01A8EA32C4E
:101B6000B22CCD84DE8473018201298139894A89AE
:101B70005B896C897D898E899F890E948D24298744
:101B80003A874B875C8789859A85AB85BC850697A4
:101B9000A105B10520F4F6E0AF2EB12C0FC0E98409
:101BA000FA840B851C8529E0E21627E0F206010580
:101BB0001105D0F078E0A72EE7E0BE2EC12CD12C85
:101BC000E12CF12C00E010E0298139894A895B89F8
:101BD0006C897D898E899F890E948D24322E232EC7
:101BE0004D875E873B012C01A32CB22CCD84DE8473
:101BF00073018201298139894A895B896C897D89D0
:101C00008E899F890E948B244901B42FA52FF62F1E
:101C1000E72F888F998F05E00E94FA245401CB2E7C
:101C2000DA2EEF2EFE2E088D198D0E943A2505E042
:101C30000E94FA24088D0E94312505E00E94FA24B2
:101C4000088D0E943A25288F398F4A01B62FA72F79
:101C5000F82FE92F6B2F7A2F8F2F9E2F05E00E94F0
:101C6000FA2459016A017B018C01288D398DA40168
:101C70006B2F7A2F8F2F9E2F0E943125A32CB22CF1
:101C8000CD84DE84730182010E948D24C22ED32E66
:101C9000E42EF52EC114D104E104F104F9F4812CF1
:101CA000912C5401839420C081E08A8F58CFAF8556
:101CB000B8891D921D921D921C921397FD011482EA
:101CC000158216821782C12CD12C7601C3941896E6
:101CD000CD92DD92ED92FC921B9722C088248A94CB
:101CE000982C8FE0A82EB12CFA8DF13009F0F5CEAA
:101CF000EF85F88910821182128213821482158274
:101D00001682178281E090E0A0E0B0E080879187A2
:101D1000A287B387232D322D4D855E85B301C20185
:101D20006A960FB6F894DEBF0FBECDBFDF91CF919C
:101D30001F910F91FF90EF90DF90CF90BF90AF90E9
:101D40009F908F907F906F905F904F903F902F90DB
:101D50000895DF92EF92FF920F931F93CF93DF933B
:101D6000FC01E080F18002811381D481C581B681BC
:101D7000D7809701A8016D2F7C2F8B2F9D2D355378
:101D80004C40510961097109810991092F3F344380
:101D90004C405105610571058105910509F098F4E4
:101DA0009701A8016D2F7C2F8B2F9D2D07E00E949E
:101DB000FA2420833183428353836483758386832B
:101DC000978387E0FDC09701A8016D2F7C2F8B2F93
:101DD0009D2D3A56484151096109710981099109BE
:101DE0002F3F39464841510561057105810591052F
:101DF00009F098F49701A8016D2F7C2F8B2F9D2D52
:101E000006E00E94FA242083318342835383648353
:101E100075838683978386E0D3C09701A8016D2FD1
:101E20007C2F8B2F9D2D345D404351096109710931
:101E3000810991092F3F334D4043510561057105DB
:101E40008105910509F098F49701A8016D2F7C2F69
:101E50008B2F9D2D05E00E94FA242083318342833D
:101E60005383648375838683978385E0A9C0970134
:101E7000A8016D2F7C2F8B2F9D2D385A414651097B
:101E800061097109810991092F3F374A414651057E
:101E9000610571058105910509F098F49701A80184
:101EA0006D2F7C2F8B2F9D2D04E00E94FA24208320
:101EB000318342835383648375838683978384E06D
:101EC0007FC09701A8016D2F7C2F8B2F9D2D305542
:101ED000434C510961097109810991092F3F3F4420
:101EE000434C5105610571058105910509F098F490
:101EF0009701A8016D2F7C2F8B2F9D2D03E00E9451
:101F0000FA242083318342835383648375838683D9
:101F1000978383E055C09701A8016D2F7C2F8B2FED
:101F20009D2D305A46485140610971098109910936
:101F30002F3F3F4946485140610571058105910594
:101F400009F098F49701A8016D2F7C2F8B2F9D2D00
:101F500002E00E94FA242083318342835383648306
:101F600075838683978382E02BC09701A8016D2F2C
:101F70007C2F8B2F9D2D30544D40534061097109AA
:101F8000810991092F3F3F434D4053406105710541
:101F90008105910509F098F49701A8016D2F7C2F18
:101FA0008B2F9D2D01E00E94FA24208331834283F0
:101FB0005383648375838683978381E001C080E0C7
:101FC000DF91CF911F910F91FF90EF90DF900895D7
:101FD0000F931F93CF938B01C0E1C80F8C2F0E94EA
:101FE00069090115110511F48F7D04C00130110537
:101FF00009F48062682F8C2FCF911F910F910C9460
:102000004F092F923F924F925F926F927F928F92E1
:102010009F92AF92BF92CF92DF92EF92FF920F9377
:102020001F93CF93DF93CDB7DEB7AA970FB6F8947F
:10203000DEBF0FBECDBF622E298F732E3A8F4B8F1E
:102040005C8F6D8F7E8F8F8F98A319A708A7930140
:102050002F3F34434C4051056105710581059105C1
:1020600009F050F4198E85E38A8F8CE08B8F1C8EDB
:102070001D8E1E8E1F8E18A2298D3A8D4B8D5C8D64
:102080006D8D7E8D8F8D98A12115304A4C4A594B0C
:10209000634071058105910569F060F0198E80EA51
:1020A0008A8F8CEA8B8F89EB8C8F83E08D8F1E8ECD
:1020B0001F8E18A2CE0149960E94A90E8AA7798C7C
:1020C000BA8DAB8DFC8DED8D6E8C5F8C48A0272D6D
:1020D0003B2F4A2F5F2F6E2F762D852D942D2F3F6E
:1020E00005ED300701E140070EE7500703E0600708
:1020F00071058105910511F008F081C09E01235FF3
:102100003F4F4901A12CECE3BE2EF3E5CF2EACE40A
:10211000DA2E10E1E12EF12C00E010E0272D3B2F0C
:102120000E94970C88A599A58130910559F18230BC
:10213000910509F440C0892B09F05DC3898D809316
:102140000F048A8D809310048B8D809311048C8DE5
:10215000809312048D8D809313048E8D80931404CC
:102160008F8D8093150488A18093160480E019A2B6
:10217000212C5CE3352E63E5462E9CE49CA3E0E134
:10218000EDA344C3898D809317048A8D809318042E
:102190008B8D809319048C8D80931A048D8D809380
:1021A0001B048E8D80931C048F8D80931D0488A149
:1021B00080931E0420C3898D80931F048A8D809391
:1021C00020048B8D809321048C8D809322048D8D2F
:1021D000809323048E8D809324048F8D8093250417
:1021E00088A18093260480E019A2212C3CE3332EA1
:1021F00043E5442E1CE41CA320E12DA307C3CE011C
:102200000D964C01A12CB12CC12CD12CE12CF12C20
:1022100000E010E0272D3B2F4A2F5F2F6E2F762DE9
:10222000852D942D0E94970CE8A5F9A5E130F105C4
:1022300009F450C0E230F10509F492C1EF2B09F026
:102240000BC3298D3A8D4B8D5C8D6D8D7E8D00E09D
:1022500010E08F8D98A10E94970C1901442E5CA369
:102260006DA3772E582E692E60E070E080E090E03C
:102270000E94E80F2092FF03309200044092010474
:102280001CA1109302042DA1209303047092040456
:102290005092050460920604898D80930F048A8D04
:1022A000809310048B8D809311048C8D8093120485
:1022B0008D8D809313048E8D809314048F8D809365
:1022C000150488A18093160481E031E039A31BA294
:1022D0001AA29FC210912F04B98DAA8DFB8DEC8D8F
:1022E0000D8D09A30E8D0AA30F8D0EA308A10FA3B8
:1022F000123009F073C02B2F3A2F4F2F5E2F69A198
:102300007AA18EA1902F30584A4156406109710937
:10231000810991092F37304E424758496240710573
:102320008105910569F160F1A0901F04B09020042F
:10233000C0902104D0902204E0902304F090240463
:1023400000912504109126042B2F3A2F4F2F5E2F3A
:1023500069A17AA18EA19FA10E94432589F01092C4
:102360001704109218041092190410921A04109273
:102370001B0410921C0410921D0410921E046CC2C7
:1023800020900704309008044090090420910A042A
:102390002CA330910B043DA370900C0450900D04BD
:1023A00060900E04CE010D964C015101C42CD22E2A
:1023B000E32EF72C052D162D2B2F3A2F4F2F5E2FA6
:1023C00069A17AA18EA19FA10E94970C61E070E0A3
:1023D00081E090E00E94E80F19A235C02093070425
:1023E000309308044093090450930A0460930B044B
:1023F00070930C0480930D0490930E048E01035F80
:102400001F4F4801A12CB12CC12CD12CE12CF12C57
:1024100000E010E02B2F3A2F4F2F5E2F69A17AA1F9
:102420008EA19FA10E94970C1901442E5CA36DA35D
:10243000772E582E692E61E070E081E090E00E94D6
:10244000E80F11E019A3298D3A8D4B8D5C8D6D8DB0
:102450007E8D8F8D98A130584A415640610971098F
:10246000810991092F37304E424758496240710522
:102470008105910509F008F457C081E080932F048D
:1024800020911F0430912004409121045091220496
:102490006091230470912404809125049091260476
:1024A000A0E00E944C2509F442C08FE194E00E9414
:1024B000A90E8AA7A0900704B0900804C090090450
:1024C000D0900A04E0900B04F0900C0400910D04ED
:1024D00010910E0420911F0430912004409121049A
:1024E000509122046091230470912404CE0101963E
:1024F0004C0180912504909126040E94970C1F9214
:102500008AA4A12CC980DA80EB80FC800D811E8119
:102510002F81388549855A856B857C8582E090E0DE
:102520000E94BC0B0F9003C088E080932F04898D1C
:10253000809317048A8D809318048B8D80931904DF
:102540008C8D80931A048D8D80931B048E8D8093C7
:102550001C048F8D80931D0488A180931E0445C1A7
:1025600070902F04B98DAA8DFB8DEC8D0D8D09A374
:102570001E8D1AA30F8D0EA318A11FA301E07012C8
:1025800073C02B2F3A2F4F2F5E2F69A17AA18EA1F6
:10259000912F30584A4156406109710981099109CA
:1025A0002F37304E424758496240710581059105E9
:1025B00069F160F1A0901F04B0902004C090210444
:1025C000D0902204E0902304F0902404009125048C
:1025D000109126042B2F3A2F4F2F5E2F69A17AA13D
:1025E0008EA19FA10E94432589F010921F04109292
:1025F00020041092210410922204109223041092BD
:10260000240410922504109226042AC12090070465
:10261000309008044090090420910A042CA33091C2
:102620000B043DA370900C0450900D0460900E04B8
:10263000CE010D964C015101C42CD22EE32EF72C65
:10264000052D162D2B2F3A2F4F2F5E2F69A17AA122
:102650008EA19FA10E94970C61E070E082E090E063
:102660000E94E80F19A235C0209307043093080494
:102670004093090450930A0460930B0470930C0474
:1026800080930D0490930E048E01035F1F4F480149
:10269000A12CB12CC12CD12CE12CF12C00E010E0AC
:1026A0002B2F3A2F4F2F5E2F69A17AA18EA19FA1C8
:1026B0000E94970C1901442E5CA36DA3772E582E0F
:1026C000692E61E070E082E090E00E94E80F11E086
:1026D00019A3298D3A8D4B8D5C8D6D8D7E8D8F8DDF
:1026E00098A130584A415640610971098109910900
:1026F0002F37304E42475849624071058105910598
:1027000009F008F457C082E080932F042091170449
:10271000309118044091190450911A0460911B04DF
:1027200070911C0480911D0490911E04A0E00E94F1
:102730004C2509F442C087E194E00E94A90E8AA7C3
:10274000A0900704B0900804C0900904D0900A0437
:10275000E0900B04F0900C0400910D0410910E0415
:1027600020911704309118044091190450911A04D3
:1027700060911B0470911C04CE0101964C01809164
:102780001D0490911E040E94970C1F928AA4A12CF4
:10279000C980DA80EB80FC800D811E812F81388515
:1027A00049855A856B857C8581E090E00E94BC0B51
:1027B0000F9003C088E080932F04898D80931F04BD
:1027C0008A8D809320048B8D809321048C8D80933F
:1027D00022048D8D809323048E8D809324048F8D0D
:1027E0008093250488A18093260481E0E1E0F0E055
:1027F000FBA3EAA30EC080E019A2212C9CE3392E92
:1028000023E5422EFCE4FCA300E10DA3712C512C26
:10281000612C8F938AA4A82ECD84DE84EF84F8885F
:1028200009891A892B893C894D895E896F89788D40
:1028300088A599A50E94BC0B0F9019A1113079F4BD
:102840000AA11BA19101442D5CA16DA1772D852DBD
:10285000962D0E94D10903C07724739401C0712C76
:10286000872DAA960FB6F894DEBF0FBECDBFDF91BD
:10287000CF911F910F91FF90EF90DF90CF90BF907D
:10288000AF909F908F907F906F905F904F903F9010
:102890002F900895DF92EF92FF920F931F93CF93A3
:1028A000DF937C018B01EA014617570720F4812F43
:1028B0008A01C62FD82F67E871E0C7010E94CA03BA
:1028C0008091EB039091EC0308171907E0F48C1743
:1028D0009D0708F4EC01E091E703F091E803EC0FA9
:1028E000FD1FD08010826091E7037091E803600FB4
:1028F000711FC7010E949703E091E703F091E8037D
:10290000EC0FFD1FD082C701DF91CF911F910F9176
:10291000FF90EF90DF90089580E480937C00809199
:102920007A00806480937A0080917A0086FDFCCFE3
:10293000809178002091790090E0922B08958F92F9
:102940009F92AF92BF920F931F93CF93DF93CDB718
:10295000DEB7A1970FB6F894DEBF0FBECDBF19A2A8
:10296000423008F44AE08E010F5D1F4F842E912CF7
:10297000A12CB12CA50194010E948023E62FB9015E
:10298000CA0101501109EA3014F4E05D01C0E95CAC
:10299000D801EC93232B242B252B61F7B8018FE969
:1029A00093E00E94DF03A1960FB6F894DEBF0FBE3E
:1029B000CDBFDF91CF911F910F91BF90AF909F90AE
:1029C0008F900895E0919F03F091A0030190F08112
:1029D000E02D682F8FE993E00994643008F063E0FC
:1029E0009091B203691710F06FEF690FE62FF0E0D6
:1029F000E156FC4F9489682F690F60688FE993E076
:102A00000C940807CF92DF92EF92FF92CF93DF935F
:102A10006C01990FEE08FF08F7FE17C08DE20E94C7
:102A2000E214EC0166277727CB016C197D098E092A
:102A30009F094AE00E949F148C0F9D1FDF91CF9148
:102A4000FF90EF90DF90CF9008954AE0C701B60164
:102A5000DF91CF91FF90EF90DF90CF900C949F1477
:102A6000FC018091BB039091BC03892B21F421E0F0
:102A7000309749F413C08091B7039091B803309711
:102A800031F421E0FC018081882341F006C0BF01C0
:102A90000E94712721E0892B09F020E0822F089500
:102AA000CF93DF93CDB7DEB7E2970FB6F894DEBFD2
:102AB0000FBECDBF789484B5826084BD84B581603B
:102AC00084BD85B5826085BD85B5816085BD8091F9
:102AD0006E00816080936E00109281008091810071
:102AE0008260809381008091810081608093810069
:102AF000809180008160809380008091B10084602B
:102B00008093B1008091B00081608093B00080918B
:102B10007A00846080937A0080917A00826080934A
:102B20007A0080917A00816080937A0080917A00A7
:102B3000806880937A001092C100E0910603F091C2
:102B4000070382E08083E0910603F091070310827F
:102B5000E0910203F09103031082E0910403F091ED
:102B6000050380E1808310920E03E0910A03F09147
:102B70000B0386E08083E0910803F09109038081D4
:102B800080618083E0910803F0910903808188606F
:102B90008083E0910803F09109038081806880833D
:102BA000E0910803F091090380818F7D808362E0CA
:102BB0008FE993E00E94670868E270E087EE93E097
:102BC0000E940F0361E085E00E94940461E08AE0C6
:102BD0000E94940461E08BE00E94940461E08CE028
:102BE0000E94940461E08DE00E94940461E08FE013
:102BF0000E94940461E080E10E94940461E081E11C
:102C00000E949404809168008460809368008091A1
:102C10006D008C6080936D00789480E090E00E945D
:102C2000BF22809305028A3FF1F06AEF69831A821E
:102C300080E090E06FA70E94BF226AEF681721F042
:102C400080E090E00E94C7226A8181E090E06FA757
:102C50000E94BF226FA5681721F081E090E00E94DA
:102C6000C7220E9423090E940A09FC0180819181E8
:102C7000A281B3818093F2029093F302A093F402B5
:102C8000B093F5028CEE9DE9A2E0B0E080932A04B7
:102C900090932B04A0932C04B0932D0410928702E0
:102CA000109286021092D0021092F1021092CE027F
:102CB00081E08093CD021092A80261E082E10E943F
:102CC0004E0461E083E10E944E048091B9008E7F42
:102CD0008093B9008091B9008D7F8093B90088E41A
:102CE0008093B80085E48093BC0062E987EB0E9482
:102CF0004F0960E880E10E944F0960E881E10E948D
:102D00004F0960E882E10E944F096CE080E10E9477
:102D10004F096CE081E10E944F096CE082E10E9462
:102D20004F0960E281EB0E944F0960E881EB0E944D
:102D30004F0900E010E020E03CE343E55CE460E1A3
:102D400070E080E090E00E94D109809100019091B4
:102D50000101A0910201B0910301BC01CD0132E05B
:102D6000660F771F881F991F3A95D1F724E630E048
:102D700040E050E00E9420240E94011080E10E9467
:102D800069098C7F682F626080E10E944F0940E4EE
:102D9000842E42E4942E4FE0A42EB12C0E943107E1
:102DA0004090010250900202609003027090040271
:102DB000411451046104710409F4C6C0C090F801C3
:102DC000D090F901E090FA01F090FB0160910702C8
:102DD000709108028091090290910A02A701960160
:102DE0000E94A223C701B6010E945C23A70196019D
:102DF0000E94A223C701B6010E945C23A70196018D
:102E00000E94A223240D351D461D571DC701B60182
:102E10000E945C236093070270930802809309026A
:102E200090930A021AA619A61CA61BA61EA61DA6EA
:102E30002AE0AE014F5F5F4F0E945421BE016F5FD9
:102E40007F4FCE0189960E9497038DA59EA50B9773
:102E500078F51CA21BA21EA21DA218A61FA24AE062
:102E6000BE016F5F7F4F80E090E00E944921BE016C
:102E70006F5F7F4FCE0183960E9497034DA55EA59D
:102E800069A57AA5CE0183960E943603811104C0FC
:102E9000CE0183960E946403BE016D5D7F4FCE011B
:102EA00089960E94AE03CE0183960E94C503CDCFC2
:102EB0006EE471E0CE0101960E94CA034DA55EA5A5
:102EC00069A57AA5CE0101960E943603811104C03E
:102ED000CE0101960E94640341E050E06FEA71E088
:102EE000CE0101960E943603882311F40C94D51F5D
:102EF000BE016F5F7F4FCE0189960E94AE03CE0167
:102F000001960E94C50380910002813019F40E944D
:102F100031070EC04DA55EA569A57AA586EF92E0A2
:102F20000E949E0063E270E080E090E00E94D00486
:102F300010920102109202021092030210920402F7
:102F4000CE0189960E94C50361E571E086EF92E0AB
:102F50000E94F40386EF92E00E94690162E370E050
:102F600080E090E00E94D00486EF92E00E94EB00A7
:102F7000892BD9F580910602811109C061E08FE9A2
:102F800093E00E9408078BE39FE10197F1F760E06F
:102F900080E00E94ED1465E571E08FE993E00E9406
:102FA000F40364EF71E080E090E00E94D00461E0FF
:102FB00080E00E94ED1466E671E08FE993E00E94E4
:102FC000F40368EE73E080E090E00E94D00461E0DA
:102FD00080E00E94ED1467E771E08FE993E00E94C2
:102FE000F40381E080930602AFCF0E940B074DE00F
:102FF00050E062E070E0CE0101960E944A14BE01EA
:103000006F5F7F4F8FEC93E00E94D602CE01019656
:103010000E94C5038FEC93E00E94CB0260930001F5
:1030200070930101809302019093030180912E021D
:103030008130A1F480913402813081F480911602B4
:1030400090911702A0911802B0911902809300018B
:1030500090930101A0930201B0930301C09000017D
:10306000D0900101E0900201F0900301C0920702AC
:10307000D0920802E0920902F0920A024EE150E07A
:103080006DE170E0CE0101960E944A14BE016F5FAF
:103090007F4F89EC93E00E94D602CE0101960E94F8
:1030A000C50389EC93E00E94CB0260932C0248E1B7
:1030B00050E067E170E0CE0101960E944A14BE0123
:1030C0006F5F7F4F8BED93E00E94D602CE01019699
:1030D0000E94C5038BED93E00E94CB0260932B020C
:1030E00049E150E068E170E0CE0101960E944A1487
:1030F000BE016F5F7F4F85ED93E00E94D602CE0147
:1031000001960E94C50385ED93E00E94CB02609377
:103110002A0241E150E06DE070E0CE0101960E948C
:103120004A14BE016F5F7F4F83EC93E00E94D6028A
:10313000CE0101960E94C50383EC93E00E94CB026E
:1031400070930C0260930B0242E150E061E170E089
:10315000CE0101960E944A14BE016F5F7F4F87EB3C
:1031600093E00E94D602CE0101960E94C50347E17A
:1031700050E062E170E0CE0101960E944A14BE0167
:103180006F5F7F4F8DEB93E00E94D602CE010196D8
:103190000E94C5038DEB93E00E94CB026093260250
:1031A0007093270280932802909329024DE150E00A
:1031B0006CE170E0CE0101960E944A14BE016F5F7F
:1031C0007F4F81EE93E00E94D602CE0101960E94CD
:1031D000C50381EE93E00E94CB026093340267E85E
:1031E00071E087EE93E00E94970380913602909100
:1031F0003702A0913802B0913902C816D906EA0602
:10320000FB0609F49BC0D701C60180549244AF402D
:10321000B10980389448AE41B10518F415B880EA78
:1032200086C0D701C601805C964CAD42B10980389A
:103230009448AE41B10520F484E085B980E577C0BB
:10324000D701C60180549B44AC44B109803C964CE4
:10325000AD42B10520F488E085B988E268C0D701A5
:10326000C6019251AA47B10981159940AD43B105F4
:1032700020F48CE085B98EE15AC0D701C6019B517C
:10328000A74BB10981159940AD43B10520F480E108
:1032900085B984E14CC0D701C6019452A44FB1094D
:1032A000803C964CAD42B10520F484E185B981E1C2
:1032B0003EC0D701C601805C9A4EA142B140803C1D
:1032C000964CAD42B10520F488E185B98FE02FC05E
:1032D000D701C6018058914BAF44B14080349B4424
:1032E000AC44B10520F48CE185B98CE020C0D70155
:1032F000C601805C9C4FAB49B14080349D45A64CD3
:10330000B10520F480E285B98AE011C0FAE5DF1A40
:10331000F2E6EF0AF2E0FF0A21E4C2162DE5D2063A
:1033200026ECE206F10428F484E285B986E0809375
:10333000300260E070E0CB010E94D00480910B026B
:1033400090910C02009729F481E090E0A0E0B0E0B9
:1033500068C08130910529F48AE090E0A0E0B0E0F7
:1033600060C0883EA3E09A0729F482E390E0A0E0E1
:10337000B0E057C08A30910529F484E690E0A0E0DF
:10338000B0E04FC0893EA3E09A0729F48AEF90E0AD
:10339000A0E0B0E046C0823FA3E09A0729F484EFA2
:1033A00091E0A0E0B0E03DC08B30910529F488EEBB
:1033B00093E0A0E0B0E035C0833FB3E09B0729F481
:1033C00088E893E1A0E0B0E02CC08C34A4E09A0738
:1033D00029F488E293E2A0E0B0E023C084369105AE
:1033E00029F480E197E2A0E0B0E01BC085369105AA
:1033F00029F480EA96E8A1E0B0E013C08E3691058A
:1034000049F48092F8019092F901A092FA01B092E9
:10341000FB010FC08F36910561F480E896E9A8E9B9
:10342000B0E08093F8019093F901A093FA01B09372
:10343000FB0160E070E0CB010E94D0040E948C147C
:103440000E948C147C016AE070E080E090E00E94B1
:10345000D0040E948C140E948C14092E000CAA0B1C
:10346000BB0BA7010F2C000C660B770B8C019D0189
:103470000D5F1F4F2F4F3F4F0417150726073707C4
:1034800064F00397A109B109481759076A077B0738
:1034900024F0F0921002E0920F0280910F029091BE
:1034A00010028538A3E09A07CCF020910E0221117A
:1034B0000DC010920D021092000210922D02109277
:1034C000250260E081E10E944E04BCC0213069F415
:1034D00010920D0281E080932502B4C083329105E1
:1034E00024F420910D02213099F79C0124523109D6
:1034F0002633310518F520910D0210910E0221118D
:103500000EC011110CC061E081E10E944E0481E007
:1035100080930E028093250280930D0293C0113098
:1035200069F421110BC060E081E10E944E04109209
:103530000E021092250210930D0284C09C012B559F
:1035400031092C32310550F420910D02211103C0B4
:1035500068E871E00FC0213009F474C09C0128585C
:10356000310926333105A8F420910D0221110EC036
:103570006EE871E086EF92E00E94F40381E08093B0
:103580000D026EE170E080E090E03CC0213009F473
:1035900059C09C012F5B31092C32310550F4209128
:1035A0000D02211103C064E971E00FC0213009F45C
:1035B00049C09C012C5E31092C32310580F42091E8
:1035C0000D0221110AC068E971E086EF92E00E94C5
:1035D000F40381E080930D0211C0213099F19C0128
:1035E000295131402D31310590F420910D022111E6
:1035F0000CC081E080930D0280932D0268E270E0A0
:1036000080E090E00E94D0041DC02130D9F09C01E0
:10361000275331402D31310560F420910D022111E5
:1036200006C081E080930D0280930002E7CF213035
:1036300049F0875D9140833B910520F480910D0214
:10364000882379F360E070E0CB010E94D0041091F0
:103650002502113081F480911102813061F061E026
:1036600081E10E944E046CE971E086EF92E00E94D5
:10367000F4031093110280912502811110C08091F2
:103680001102813061F460E081E10E944E0460EA41
:1036900071E086EF92E00E94F40310921102109103
:1036A0003402113011F461E003C0111104C060E074
:1036B00081E10E944E04809135028F5F8093350234
:1036C0008A3009F059C0113009F456C01092350201
:1036D00064EA71E086EF92E00E94F40386EF92E0E4
:1036E0000E94690164E670E080E090E00E94D004EE
:1036F0000E940B0745E050E064E070E0CE010196C7
:103700000E944A14BE016F5F7F4F8DEE93E00E94CE
:10371000D602CE0101960E94C5038DEE93E00E9471
:10372000CB02162F6093240267E871E087EE93E0E6
:103730000E94970310921202109213021092140228
:1037400010921502111102C061E003C0113031F472
:1037500060E08FE00E944E0460E00BC0123011F474
:1037600061E003C0133041F460E08FE00E944E043A
:1037700061E080E10E944E04809133028F5F80936C
:103780003302853009F041C0809134028130E9F183
:10379000109233026AEA71E086EF92E00E94F4032D
:1037A00086EF92E00E94690166E470E080E090E0BC
:1037B0000E94D0040E940B0748E050E065E070E0F2
:1037C000CE0101960E944A14BE016F5F7F4F8DEEBD
:1037D00093E00E94D602CE0101960E94C5038DEEB1
:1037E00093E00E94CB0270931F0260931E0267E871
:1037F00071E087EE93E00E949703109212021092FC
:1038000013021092140210921502809132028F5FFF
:10381000809332028431D9F51092320261EB71E06B
:1038200086EF92E00E94F40386EF92E00E94690125
:1038300062E370E080E090E00E94D0040E940B07F9
:1038400045E050E064E070E0CE0101960E944A1429
:10385000BE016F5F7F4F8DEE93E00E94D602CE01D6
:1038600001960E94C5038DEE93E00E94CB02609307
:103870002E0267E871E087EE93E00E9497031092B2
:1038800012021092130210921402109215028091EB
:103890003402813009F03FC067EB71E086EF92E0BF
:1038A0000E94F40386EF92E00E94690162E370E0F7
:1038B00080E090E00E94D0040E940B074DE050E0B1
:1038C00064E070E0CE0101960E944A14BE016F5F71
:1038D0007F4F8DEE93E00E94D602CE0101960E94AA
:1038E000C5038DEE93E00E94CB02609316027093A5
:1038F0001702809318029093190267E871E087EE2F
:1039000093E00E94970310921202109213021092F9
:103910001402109215028091000260E0813009F4D7
:1039200096C183E00E94ED14609100017091010145
:103930008091020190910301A50194010E94A223AC
:103940002A30310558F480E22FA738AB49AB5AAB87
:103950000E94E2145AA949A938A92FA5CA01B901A0
:10396000882799274AE00E949F148EE20E94E21461
:103970006091000170910101809102019091030119
:10398000A50194010E94A22328EE33E040E050E01C
:103990000E94A223790124363105B0F480E32FA7D9
:1039A00038AB49AB5AAB0E94E2142FA538A949A9FC
:1039B0005AA9EAE0EE16F10438F480E30E94E2141A
:1039C0005AA949A938A92FA5CA01B9018827992759
:1039D0004AE00E949F148EE20E94E214609100016E
:1039E00070910101809102019091030128EE33E072
:1039F00040E050E00E94A2236B017C018B01643601
:103A0000710548F480E30E94E2140A30110518F4AD
:103A100080E30E94E214C701B601882799274AE093
:103A20000E949F146BEB71E08FE993E00E94F40316
:103A30008091250281110DC080913402811109C04D
:103A400060E00E94ED146FEB71E08FE993E00E945B
:103A5000F40380912502813021F08091340281307D
:103A600081F465E871E08FE993E00E94F40360E07F
:103A700080E00E94ED1463EC71E08FE993E00E9416
:103A8000F40361E084E00E94ED1464E871E08FE9E2
:103A900093E00E94F40380912402811109C061E047
:103AA0000E94ED1467EC71E08FE993E00E94F4034B
:103AB00080912402813051F461E080E00E94ED1495
:103AC0006CEC71E08FE993E00E94F4038091240292
:103AD000823051F461E080E00E94ED1461ED71E00C
:103AE0008FE993E00E94F40380912402833051F423
:103AF00061E080E00E94ED1466ED71E08FE993E0F3
:103B00000E94F4032FB7F8948091FC019091FD017D
:103B1000A091FE01B091FF012FBF40912002509172
:103B200021026091220270912302841B950BA60B47
:103B3000B70B853F9140A105B10508F4BAC061E01B
:103B400087E00E94ED146BED71E08FE993E00E9435
:103B5000F40380911E0290911F028D3891050CF59F
:103B600044976CE070E00E946C23161617062CF444
:103B700070931D0260931C0204C010921D021092EB
:103B80001C0261E08AE00E94ED1480911C02909179
:103B90001D020E94021562E871E08FE993E00E9425
:103BA000F40360911E0270911F026D387105DCF103
:103BB00089E090E090931D0280931C026658710981
:103BC000072E000C880B990B0E94C62120E030E0E4
:103BD00040E05FE30E9401220E94262370931B02B3
:103BE00060931A0261E08AE00E94ED1489E090E09F
:103BF0000E94021561E08BE00E94ED146FED71E010
:103C00008FE993E00E94F40380911A0290911B02C5
:103C10000E94021561EE71E08FE993E00E94F403C7
:103C200080E20E94E2142FB7F8948091FC019091F9
:103C3000FD01A091FE01B091FF012FBF80932002F2
:103C400090932102A0932202B093230232C080E01D
:103C50000E94ED1464EE71E08FE993E00E94F4039A
:103C600061E080E00E94ED1468E771E08FE993E085
:103C70000E94F40361E085E00E94ED14C090F2021E
:103C8000D090F302E090F402F090F502F7FE0CC041
:103C90008DE20E94E21466277727CB016C197D091B
:103CA0008E099F094AE003C04AE0C701B6010E949D
:103CB0009F148091000190910101A0910201B091A7
:103CC000030181349244AF40B10544F48092000175
:103CD00090920101A0920201B09203018091000133
:103CE00090910101A0910201B0910301803C9243A7
:103CF000AA40B34064F080EC92E3AAE0B3E0809382
:103D0000000190930101A0930201B09303019091EF
:103D10002C02809134029430B9F48130A9F480915E
:103D2000000190910101A0910201B0910301885F0F
:103D30009A42A109B1098093000190930101A093D7
:103D40000201B093030123C081111EC080912B0298
:103D5000811105C080912A0281112DC108C08130D6
:103D600009F062C080912A02813009F028C1809157
:103D7000000190910101A0910201B09103018852CC
:103D80009342A109B10948C0813009F04DC080912A
:103D90002B02811149C080912A02813009F044C070
:103DA0008FED91E00E9430158823E1F040910001F1
:103DB00050910101609102017091030180912602EE
:103DC00090912702A0912802B0912902840F951F9B
:103DD000A61FB71F8093000190930101A0930201D9
:103DE000B093030185EF91E00E9430158823E1F044
:103DF0008091000190910101A0910201B091030115
:103E00004091260250912702609128027091290268
:103E1000841B950BA60BB70B8093000190930101B7
:103E2000A0930201B0930301809131028F5F883C1F
:103E300019F08093310202C010923102C09000014B
:103E4000D0900101E0900201F090030180913602D0
:103E500090913702A0913802B0913902C816D90664
:103E6000EA06FB0621F4809100028130F9F480918A
:103E7000F2029091F302A091F402B091F5028C0D40
:103E80009D1DAE1DBF1DBC01CD0122E0660F771F39
:103E9000881F991F2A95D1F724E630E040E050E0D2
:103EA0000E94202400E010E00E94011030903002B7
:103EB00080912F02381671F180912E0281112AC053
:103EC0001092340283E00E946909682F6B7F83E0BF
:103ED0000E944F098091F2029091F302A091F402A6
:103EE000B091F5028C0D9D1DAE1DBF1DBC01CD0115
:103EF000685B7E488F4F9F4F24E630E040E050E003
:103F00000E94202402E010E00E94011030922F0253
:103F10001092310280913102873C41F483E00E948B
:103F20006909682F646083E00E944F0980912D0227
:103F3000813029F583E00E946909682F6D7F83E055
:103F40000E944F098091F2029091F302A091F40235
:103F5000B091F5028C0D9D1DAE1DBF1DBC01CD01A4
:103F6000685D7C4D8F4F9F4F24E630E040E050E08D
:103F70000E94202401E010E00E9401100AC081117B
:103F800008C083E00E946909682F626083E00E9494
:103F90004F09C0923602D0923702E0923802F09276
:103FA00039020E948B010C94CE16CE0101960E941C
:103FB00064030C947817813009F036CFD8CE811184
:103FC00033CFC0900001D0900101E0900201F09049
:103FD0000301F8E2CF1AF3E2DF0AE108F108C09228
:103FE0000001D0920101E0920201F09203018FEDF5
:103FF00091E00E943015882309F4F4CE80912602C6
:1040000090912702A0912802B0912902C80ED91ED2
:10401000EA1EFB1EC0920001D0920101E092020153
:10402000F0920301DFCE87EB93E00E94C5038DEB96
:1040300093E00E94C50383EC93E00E94C50389ECE2
:1040400093E00E94C5038FEC93E00E94C50385EDC9
:1040500093E00E94C5038BED93E00E94C50381EEBF
:1040600093E00E94C50387EE93E00E94C5038DEEA6
:1040700093E00C94C5031F93CF93DF93E6EFF2E038
:104080001382128288EE93E0A0E0B0E084839583EF
:10409000A683B7832AE231E03183208325EC30E028
:1040A0003587248724EC30E03787268720EC30E002
:1040B000318B208B21EC30E0338B228B22EC30E0F3
:1040C000358B248B26EC30E0378B268B118E128EAD
:1040D000138E148EE3E9F3E01382128284839583B6
:1040E000A683B7838AE391E091838083E6EFF3E0D0
:1040F00018E010AF11AF11AA12AA13AA11861286E6
:1041000013861486158616861786108A118A128AD7
:10411000138A148A158A168A178A108E118E128EA7
:10412000138E148E158E168E178E10A211A212A247
:1041300013A214A215A216A217A210A611A612A6C7
:1041400013A614A615A616A617A610AA80E498E72B
:10415000ADE7B1E082AF93AFA4AFB5AFC3EFD3E0AB
:1041600082E0898383E08A8360E082E00E94940495
:1041700060E08A810E94940461E089810E944E047B
:1041800061E08A810E944E04188267E871E08DEE3A
:1041900093E00E94CA0367E871E087EE93E00E9413
:1041A000CA0367E871E081EE93E00E94CA0367E802
:1041B00071E08BED93E00E94CA0367E871E085ED42
:1041C00093E00E94CA0367E871E08FEC93E00E94DD
:1041D000CA0367E871E089EC93E00E94CA0367E8CC
:1041E00071E083EC93E00E94CA0367E871E08DEB15
:1041F00093E00E94CA0367E871E087EB93E00E94B6
:10420000CA03EFE9F3E0138212828AE491E091831A
:10421000808389E084838FEF8583168387E087839B
:1042200086E0808785E0818784E082871386148614
:1042300015861686178661E0CF01DF91CF911F9119
:104240000C9467081F93FC0199278827BC01E89408
:1042500011911032E9F3193010F01E30C8F31B32FF
:1042600051F01D3249F4689406C00E946321610F29
:10427000711D811D911D119110531A30B0F33EF440
:1042800090958095709561957F4F8F4F9F4F1F91AF
:104290000895BB274A3031F4992322F4BDE290956A
:1042A00081959F4F0C949B21BB272A3051F4992371
:1042B00042F4BDE290958095709561957F4F8F4F48
:1042C0009F4F0C947921592F482F372F262F660F97
:1042D000771F881F991F660F771F881F991F620F0E
:1042E000731F841F951F660F771F881F991F0895DE
:1042F000BB27FA01A62F6217710581059105330BC3
:1043000030FB66F0AA27660F771F881F991FAA1F28
:10431000A21710F0A21B63953850A9F7A05DAA332D
:1043200008F0A95DA19336F7B111B1931082CA01CB
:104330000C94B421BB27FB015527AA27880F991F8E
:10434000AA1FA41710F0A41B83955051B9F7A05DC4
:10435000AA3308F0A95DA193009779F7B111B19341
:104360001192CB010C94B421DC01FC01672F7191F7
:104370007723E1F7329704C07C916D93708362914B
:10438000AE17BF07C8F30895E89409C097FB3EF441
:1043900090958095709561957F4F8F4F9F4F992392
:1043A000A9F0F92F96E9BB279395F6958795779510
:1043B0006795B795F111F8CFFAF4BB0F11F460FFD0
:1043C0001BC06F5F7F4F8F4F9F4F16C0882311F028
:1043D00096E911C0772321F09EE8872F762F05C03C
:1043E000662371F096E8862F70E060E02AF09A95D7
:1043F000660F771F881FDAF7880F9695879597F9CC
:1044000008950E9414220C9485220E94772238F08D
:104410000E947E2220F0952311F00C946E220C94C1
:10442000742211240C94B9220E94962270F3959F55
:10443000C1F3950F50E0551F629FF001729FBB279B
:10444000F00DB11D639FAA27F00DB11DAA1F649F37
:104450006627B00DA11D661F829F2227B00DA11DEA
:10446000621F739FB00DA11D621F839FA00D611D70
:10447000221F749F3327A00D611D231F849F600D91
:10448000211D822F762F6A2F11249F5750409AF0BA
:10449000F1F088234AF0EE0FFF1FBB1F661F771F46
:1044A000881F91505040A9F79E3F510580F00C9411
:1044B0006E220C94B9225F3FE4F3983ED4F38695C4
:1044C00077956795B795F795E7959F5FC1F7FE2BB1
:1044D000880F911D9695879597F9089597F99F678D
:1044E00080E870E060E008959FEF80EC089500247C
:1044F0000A941616170618060906089500240A9449
:1045000012161306140605060895092E0394000CCE
:1045100011F4882352F0BB0F40F4BF2B11F460FF5D
:1045200004C06F5F7F4F8F4F9F4F089557FD905886
:10453000440F551F59F05F3F71F04795880F97FB67
:10454000991F61F09F3F79F0879508951216130621
:104550001406551FF2CF4695F1DF08C01616170650
:104560001806991FF1CF8695710561050894089585
:10457000E894BB2766277727CB0197F90895F99927
:10458000FECF92BD81BDF89A992780B50895262F58
:10459000F999FECF1FBA92BD81BD20BD0FB6F89428
:1045A000FA9AF99A0FBE019608950E941723A59FC3
:1045B000900DB49F900DA49F800D911D112408951E
:1045C0002F923F924F925F926F927F928F929F9223
:1045D000AF92BF92CF92DF92EF92FF920F931F9311
:1045E000CF93DF93CDB7DEB7CA1BDB0B0FB6F894C2
:1045F000DEBF0FBECDBF09942A88398848885F8402
:104600006E847D848C849B84AA84B984C884DF8072
:10461000EE80FD800C811B81AA81B981CE0FD11D56
:104620000FB6F894DEBF0FBECDBFED010895A29F77
:10463000B001B39FC001A39F700D811D1124911D76
:10464000B29F700D811D1124911D08950E942D238C
:104650006894B1110C94B92208950E949E2288F0AA
:104660009F5798F0B92F9927B751B0F0E1F0660F36
:10467000771F881F991F1AF0BA95C9F714C0B13077
:1046800091F00E94B822B1E008950C94B822672FEF
:10469000782F8827B85F39F0B93FCCF386957795A6
:1046A0006795B395D9F73EF490958095709561958F
:1046B0007F4F8F4F9F4F0895DB018F939F930E94F1
:1046C000D522BF91AF91A29F800D911DA39F900D08
:1046D000B29F900D1124089597FB072E16F40094B5
:1046E00007D077FD09D00E94582507FC05D03EF47D
:1046F000909581959F4F0895709561957F4F08958E
:10470000A1E21A2EAA1BBB1BFD010DC0AA1FBB1FD5
:10471000EE1FFF1FA217B307E407F50720F0A21B47
:10472000B30BE40BF50B661F771F881F991F1A94B4
:1047300069F760957095809590959B01AC01BD01DE
:10474000CF010895052E97FB1EF400940E94B92313
:1047500057FD07D00E94802307FC03D04EF40C9431
:10476000B92350954095309521953F4F4F4F5F4F5E
:10477000089590958095709561957F4F8F4F9F4FCD
:104780000895EE0FFF1F0590F491E02D0994DF933B
:10479000CF931F930F939A9DF02D219FF00D8B9D2A
:1047A000F00D8A9DE02DF10D039FF00D029FE00DAD
:1047B000F11D4E9DE00DF11D5E9DF00D4F9DF00D24
:1047C0007F936F93BF92AF925F934F93D5010E94F7
:1047D00017238B01AC01D7010E941723EB01E80FCF
:1047E000F91FD6010E9417242F913F91D6010E94F4
:1047F0001723C60FD71FE81FF91FAF91BF910E9463
:1048000017242F913F910E941723C60FD71FE81F2F
:10481000F91FD6010E941723E60FF71F9801BE016A
:10482000CF0111240F911F91CF91DF9108950E9424
:104830001723460F571FC81FD91F08F43196089534
:1048400097FB57FF0C9430249F938F930E94302442
:104850006E1B7F0BAF91BF918A0B9B0B0895E89461
:10486000DF93CF93FC01DB010E9417237F936F93AB
:10487000E9019A01AC01BF93AF933F932F93DF01FE
:104880000E94172326F46C1B7D0B820B930B9E0159
:10489000EB01FC010E941724AF91BF912F913F9132
:1048A0000E941724BE01CF01F9012F913F91CF91B2
:1048B000DF910895689401C0E894F92FF12B12F06C
:1048C0000C948E24A0E0B0E0E8E6F4E20C94E6223A
:1048D000092E059422F40E94EA24112392F4F0E8B0
:1048E0000F26FFEFE094F09400951095B094C094DB
:1048F000D094A194BF0ACF0ADF0AEF0AFF0A0F0B78
:104900001F0B0E94992407FC0E94EA24CDB7DEB752
:10491000ECE00C940223689401C0E8948F929F927B
:10492000CF93DF930E949924DF91CF919F908F9036
:10493000089588249924F401E401B0E49F93AA2700
:104940009A158B049C04ED05FE05CF05D007A10741
:1049500098F4AD2FDC2FCF2FFE2FE92D982C892E28
:10496000982F872F762F652F542F432F322F2227F2
:10497000B85031F7BF9127C01B2EBF91BB27220F24
:10498000331F441F551F661F771F881F991F881CE0
:10499000991CEE1FFF1FCC1FDD1FAA1FBB1F8A140F
:1049A0009B04EC05FD05CE05DF05A007B10748F027
:1049B0008A189B08EC09FD09CE09DF09A00BB10B91
:1049C00021601A94E1F62EF49401AF01BE01CD01ED
:1049D000000C089560957095809590953095409560
:1049E000509521953F4F4F4F5F4F6F4F7F4F8F4FE8
:1049F0009F4F08950F93083090F0982F872F762FB0
:104A0000652F542F432F322F22270850F4CF220F27
:104A1000331F441F551F661F771F881F991F0A9554
:104A2000B2F70F91089597FB10F8169400080F93B2
:104A3000083098F00850232F342F452F562F672F1A
:104A4000782F892F902DF4CF05949795879577959A
:104A5000679557954795379527950A95AAF70F912A
:104A600008952A0D3B1D4C1D5D1D6E1D7F1D801F71
:104A7000911F08952A193B094C095D096E097F09A8
:104A8000800B910B08952A153B054C055D056E05BD
:104A90007F058007910708950024A7FD00942A1739
:104AA00030054005500560057005800590050895A6
:104AB000AA1BBB1B51E107C0AA1FBB1FA617B70744
:104AC00010F0A61BB70B881F991F5A95A9F7809560
:104AD0009095BC01CD010895CF93DF93823091056D
:104AE00010F482E090E0E0913704F091380420E087
:104AF00030E0C0E0D0E0309711F14081518148179B
:104B00005907C0F04817590761F4828193812097B3
:104B100019F09B838A832BC09093380480933704C9
:104B200026C02115310519F04217530718F49A01D0
:104B3000BE01DF01EF010280F381E02DDCCF211502
:104B4000310509F1281B390B2430310590F41296F8
:104B50008D919C9113976115710521F0FB01938351
:104B6000828304C09093380480933704FD01329609
:104B700044C0FD01E20FF31F81939193225031094C
:104B80002D933C933AC02091350430913604232B69
:104B900041F42091060130910701309336042093AF
:104BA000350420910401309105012115310541F4AE
:104BB0002DB73EB74091080150910901241B350BD8
:104BC000E0913504F0913604E217F307A0F42E1BB0
:104BD0003F0B2817390778F0AC014E5F5F4F241761
:104BE000350748F04E0F5F1F50933604409335044D
:104BF0008193919302C0E0E0F0E0CF01DF91CF918B
:104C000008950F931F93CF93DF93009709F48CC0FF
:104C1000FC013297138212820091370410913804FC
:104C20000115110581F420813181820F931F20919C
:104C30003504309136042817390779F5F093360496
:104C4000E093350471C0D80140E050E0AE17BF07D3
:104C500050F412962D913C911397AD012115310519
:104C600009F1D901F3CF9D01DA01338322836081F9
:104C70007181860F971F8217930769F4EC012881D1
:104C80003981260F371F2E5F3F4F318320838A8162
:104C90009B8193838283452B29F4F0933804E0931E
:104CA000370442C01396FC93EE931297ED0149919D
:104CB00059919E01240F351FE217F30771F480818B
:104CC0009181840F951F029611969C938E938281F9
:104CD000938113969C938E931297E0E0F0E0D801B5
:104CE00012968D919C911397009719F0F8018C0101
:104CF000F6CF8D919C9198012E5F3F4F820F931FAD
:104D000020913504309136042817390769F430971B
:104D100029F4109238041092370402C013821282D0
:104D20001093360400933504DF91CF911F910F91BA
:104D30000895A0E0B0E0EFE9F6E20C94E422EC0183
:104D4000009721F4CB010E946C25B8C0FC01E60F4E
:104D5000F71F9C0122503109E217F30708F4ACC099
:104D6000D9010D911C91119706171707B0F0053066
:104D7000110508F49FC0C80104978617970708F427
:104D800099C002501109061B170B019311936D93E3
:104D90007C93CF010E9401268DC05B01A01AB10A4D
:104DA0004C01800E911EA0913704B091380440E070
:104DB00050E0E12CF12C109709F44AC0A815B90570
:104DC000D1F56D907C901197630182E0C80ED11CE3
:104DD000CA14DB0480F1A3014A195B096A0182E06D
:104DE000C80ED11C1296BC9012971396AC91B5E0E8
:104DF000CB16D10440F0B282A38351834083D90102
:104E00006D937C930AC00E5F1F4FC301800F911FEB
:104E1000F90191838083EB2DFA2FE114F10431F035
:104E2000D7011396FC93EE93129744C0F093380485
:104E3000E09337043FC08D919C9111974817590713
:104E400008F4AC017D0112960D90BC91A02DB3CF5A
:104E5000809135049091360488159905E1F4461740
:104E60005707C8F48091040190910501009741F41F
:104E70008DB79EB74091080150910901841B950B95
:104E8000E817F907C8F4F0933604E0933504F90104
:104E9000718360830FC0CB010E946C257C01009759
:104EA00059F0A801BE010E946827CE010E94012688
:104EB000C70104C0CE0102C080E090E0CDB7DEB7EC
:104EC000EEE00C94002381E090E0F8940C948127AC
:104ED000FB01DC0102C001900D9241505040D8F717
:104EE0000895FB01DC018D91019080190110D9F327
:104EF000990B0895FB01DC0101900D920020E1F770
:104F0000089510E0C2E7D0E004C0FE010E94C12372
:0C4F10002196C337D107C9F7F894FFCFF2
:104F1C00D0B1370000003904800000020400030007
:104F2C000110030200000302010006000400060544
:104F3C000020060504000000000022019E00EB008A
:104F4C00C900DD006901000000009A026A026202D9
:104F5C004E023F023E020000000002079E00464146
:104F6C000049463B0020204E6F20636F6E6E6563D8
:104F7C0074696F6E200020202020506F776572536B
:104F8C0044522020202000202020202020202020DF
:104F9C0020202020202020005A5A53553B005A5ADA
:104FAC0053443B0042553B0042443B0054583B00A9
:104FBC0052583B005A5A50413B005A5A534D303BC1
:104FCC00005A5A53503B0046423B0020487A00524C
:104FDC00582000545820004F666620004C6F7720F4
:104FEC00004D656420004869676800536D3A002BDA
:104FFC0000644200436F7272656374696F6E2020A7
:08500C0046524551002D000041
:00000001FF
